:020000040800F2
:10000000D01300246D030008E911000879110008DD
:10001000E1110008810500087114000800000000CB
:100020000000000000000000000000009112000825
:10003000890500080000000021120008F9120008DC
:100040008B0300088B0300088B0300088B03000858
:100050008B0300088B0300088B0300088B03000848
:100060008B0300088B0300088B0300088B03000838
:100070008B0300088B0300088B0300088B03000828
:100080008B0300088B0300088B0300088B03000818
:100090008B0300088B0300088B0300088B03000808
:1000A0008B0300088B0300088B0300088B030008F8
:1000B0008B0300088B0300088B0300088B030008E8
:1000C0008B0300088B0300088B0300088B030008D8
:1000D0008B0300088B0300088B0300088B030008C8
:1000E0008B0300088B030008000000008B0300084E
:1000F0008B0300088B0300088B0300088B030008A8
:100100008B0300088B0300088B0300088B03000897
:100110008B0300088B0300088B0300088B03000887
:100120008B0300088B0300088B0300088B03000877
:100130008B0300088B0300088B0300088B03000867
:1001400000000000000000000000000000000000AF
:100150008B0300088B0300088B0300088B03000847
:100160008B0300088B0300088B0300088B03000837
:100170008B0300088B0300088B03000800000000BD
:100180008B0300088B0300088B0300088B03000817
:100190008B0300088B0300088B0300088B03000807
:1001A0008B0300088B0300088B030008000000008D
:1001B0008B0300088B0300088B0300088B030008E7
:1001C0008B0300088B030008000000000000000003
:1001D00000000000000000008B0300080000000089
:1001E000000000000000000000000000000000000F
:1001F00000000000000000008B0300088B030008D3
:100200008B0300088B030008000000008B0300082C
:100210008B0300088B0300088B0300088B03000886
:100220008B030008000000008B03000800000000A2
:100230008B0300088B030008000000008B030008FC
:100240008B0300088B0300088B0300088B03000856
:100250008B0300088B0300088B0300088B03000846
:100260008B0300088B0300088B0300088B03000836
:100270008B0300088B0300088B03000800000000BC
:100280008B0300088B0300088B0300088B03000816
:10029000000000008B0300088B0300080000000032
:1002A000000000008B0300088B0300088B0300088C
:1002B0008B0300088B0300088B0300088B030008E6
:1002C0008B0300088B0300088B03000800F002F882
:1002D00000F03CF80AA090E8000C82448344AAF1A4
:1002E0000107DA4501D100F031F8AFF2090EBAE8A2
:1002F0000F0013F0010F18BFFB1A43F0010318475A
:10030000C0300000F0300000103A24BF78C878C137
:10031000FAD8520724BF30C830C144BF04680C600B
:10032000704700000023002400250026103A28BF53
:1003300078C1FBD8520728BF30C148BF0B60704757
:100340001FB503F010F81FBD10B510BD00F0DBF8AD
:100350001146FFF7F5FF01F0C3F800F0F9F803B418
:10036000FFF7F2FF03BC00F001F900000A488047E4
:100370000A4880470A480047FEE7FEE7FEE7FEE737
:10038000FEE7FEE7FEE7FEE7FEE7FEE70548064973
:10039000064A074B70470000A105000899130008A2
:1003A000CD020008D00D0024D0130024D00F00246B
:1003B000D00F0024032A40F2308010F0030C00F02C
:1003C000158011F8013BBCF1020F624498BF11F88F
:1003D00001CB00F8013B38BF11F8013BA2F1040248
:1003E00098BF00F801CB38BF00F8013B11F00303C0
:1003F00000F05780083AC0F0088051F8043B083AF2
:1004000051F804CBA0E80810F5E7121D5CBF51F8C5
:10041000043B40F8043BAFF30080D20724BF11F83F
:10042000013B11F801CB48BF11F8012B24BF00F8A4
:10043000013B00F801CB48BF00F8012B704702F0E8
:10044000FF0343EA032242EA024200F002B84FF0FF
:10045000000200B5134694469646203922BFA0E814
:100460000C50A0E80C50B1F12001BFF4F7AF090720
:1004700028BFA0E80C5048BF0CC05DF804EB890011
:1004800028BF40F8042B08BF704748BF20F8022B54
:1004900011F0804F18BF00F8012B7047704770476C
:1004A000704710B5203AC0F00B80B1E81850A0E8B2
:1004B0001850B1E81850A0E81850203ABFF4F5AF32
:1004C0005FEA027C24BFB1E81850A0E8185044BF8E
:1004D00018C918C0BDE810405FEA827C24BF51F8FB
:1004E000043B40F8043B08BF7047D20728BF31F8EF
:1004F000023B48BF11F8012B28BF20F8023B48BF40
:1005000000F8012B7047754600F02CF8AE46050048
:100510006946534620F00700854618B020B5FFF71E
:1005200035FFBDE820404FF000064FF000074FF0C8
:1005300000084FF0000BAC46ACE8C009ACE8C009BD
:10054000ACE8C009ACE8C00921F007018D4670474E
:1005500010B50446AFF300802046BDE81040FFF719
:10056000FEBE000000487047180000240149182012
:10057000ABBEFEE72600020070470000000000004E
:10058000FEE70000000000007047000000000000CF
:10059000EFF3108072B600BFFEE70000000000001D
:1005A00044F60C00C5F60200016841F0020101604A
:1005B00050F8081C8904FBD57047000000000000BB
:1005C00040F2F450C2F200400068704700000000A2
:1005D00040F2080040F2F451C2F20040C2F2004181
:1005E00000780A68104408607047000000000000AE
:1005F00080B5032000F0D4F800F026FA44F2184148
:1006000043F28033C5F60201C0F600030A680968A8
:1006100001F00F01C2F30322595C9A5C01F01F0143
:1006200002F01F02D04040F20402C2F2004220FA5F
:1006300001F1116040F20001C2F2004108600F2098
:1006400000F00AF800281CBF012080BD00F080F8EF
:10065000002080BD00000000B0B540F20801C2F2E9
:100660000041097801B3044640F20000C2F20040A4
:100670004FF47A72B2FBF1F10068B0FBF1F000F0D8
:1006800077FD0F2C4FF001050CD858B94FF0FF3013
:1006900000222146002500F073F840F20C00C2F25F
:1006A000004004602846B0BD0120B0BD000000003D
:1006B00010B54EF6A05E4178CEF2000E90F800C064
:1006C0004EF8081CDEF8001021F00101CEF80010F1
:1006D00041684EF8041C017BC37A827A447B1B0676
:1006E00043EA0171837B41EAC241C27B41EA844112
:1006F000447A41EA4341007A41EA024141EA042155
:1007000041EA400040EA0C00CEF8000010BD0000B5
:100710004EF62450CEF20000BFF35F8F016821F443
:100720008031016000210167704700000000000077
:100730004EF6245140F00100CEF20001086708682F
:1007400040F480300860BFF34F8FBFF36F8F704766
:1007500080B582B044F2F4400022C5F60200016880
:1007600041F00201016000680F2100F002000190D9
:1007700001986FF0010000F003F802B080BD0000A6
:1007800070B514460D46064600F076FE2946224610
:1007900000F02EFD0146304600F076FE70BD0000F0
:1007A00080B500F08DFE80BDB0B544F60C05C5F6F1
:1007B000020529684907296805D401F00701081ACC
:1007C00018BF0120B0BD21F0070108432860FFF7E2
:1007D000F7FE044655F8080C800407D4FFF7F0FE36
:1007E000001BB0F57A7FF5D90120B0BD0020B0BD67
:1007F0002DE9F04381B0002800F0F48042F20008B7
:100800000446C5F200288946D8F8000000F00F0021
:1008100088420ED2D8F8000020F00F0040EA09000C
:10082000C8F80000D8F8000000F00F00484540F07C
:10083000D980206844F218474107C5F602070AD557
:1008400021693A6802F07002914204D93A6822F0B4
:1008500070021143396001070AD561697A6802F0B4
:100860007002914204D97A6822F0700211437960D3
:10087000C1060AD5A1697A6802F4E062914204D9FE
:100880007A6822F4E0621143796081060AD5E16951
:10089000BA6802F07002914204D9BA6822F070027C
:1008A0001143B96081070AD5E1683A6802F00F0286
:1008B000914204D93A6822F00F0211433960C0070F
:1008C0007ED1206881070AD5E1683A6802F00F02FC
:1008D000914204D23A6822F00F0211433960D8F8ED
:1008E000001001F00F0149450DD9D8F8001021F092
:1008F0000F0141EA0901C8F80010D8F8001001F012
:100900000F0149456ED141070AD521693A6802F0C5
:100910007002914204D23A6822F0700211433960A9
:1009200001070AD561697A6802F07002914204D227
:100930007A6822F0700211437960C1060AD5A16974
:100940007A6802F4E062914204D27A6822F4E062AA
:100950001143796080060AD5E069B96801F0700139
:10096000884204D2B96821F070010843B86000F0F1
:100970006BF8396843F28032C0F600023B68C1F37D
:10098000032103F00F03515CD25C01F01F01C8404A
:1009900002F01F0140F2040220FA01F1C2F200420B
:1009A000116040F2000140F20C02C2F20041C2F2BA
:1009B000004208601068FFF74FFE01B0BDE8F08309
:1009C000386820F47061D4E90102012841EA02018B
:1009D00039600BD003282BD002282ED157F8181CD1
:1009E000890307D4012001B0BDE8F08357F8181C33
:1009F000C905F7D557F8081C21F00701084347F847
:100A0000080CFFF7DDFD064641F2883557F8080C63
:100A1000616800F03800B0EBC10F3FF452AFFFF750
:100A2000CFFD801BA842F1D9032001B0BDE8F083BF
:100A300057F8181C8901D5D5DCE757F8181C490769
:100A4000D0D5D7E70000000044F20041C5F602010E
:100A50000869C0F3C20003280FD002282AD070BB57
:100A60000868800649F20000C0F2D03058BF7047D5
:100A70000968C1F3C101C84070478A6A886AC0F337
:100A8000051CC86ABCF1000F4B6B1DD0C3F3CC032F
:100A900000F00100584302F00302022A00EE100A9F
:100AA000B8EE400A12D0A2B90868800614D49FEDAF
:100AB000261A1EE047F64000C0F27D10704740F64F
:100AC0000010C0F23D007047002070479FED1D1AD6
:100AD0000FE09FED1B1A0CE0086849F20002C0F21B
:100AE000D032C0F3C10022FA00F001EE100AB8EED5
:100AF000411A086B9FED153A6FF35F2002EE100A62
:100B0000086BC0F34620B8EE422A013000EE032AFB
:100B100000EE10CAB7EE003AB8EE400A81EE000AC5
:100B200032EE031A20EE010A01EE100AB8EE411A65
:100B300080EE010ABCEEC00A10EE100A704700BF3A
:100B40000024744A20BCBE4B0024744C00000039C1
:100B50002DE9F04381B0F8B18046007844F20049B5
:100B6000C007C5F602095CD0D9F8100000F03801C2
:100B7000D9F82800102905D018290FD100F003005A
:100B800002280BD1D9F80000800346D5D8F804001C
:100B9000002842D1012731E00127E2E2D8F80450D1
:100BA0002DB1B5F5A02F0DD0B5F5803F10D0D9F8F7
:100BB000000020F48030C9F80000D9F8000020F4CB
:100BC000802009E0D9F8000040F48020C9F8000036
:100BD000D9F8000040F48030C9F80000FFF7F0FCBD
:100BE000002D054615D000BFD9F80000800314D4AD
:100BF000FFF7E6FC401B6428F6D9032700200028F5
:100C000000F0AF820DE000BFFFF7DAFC401B642864
:100C1000F3D8D9F800008003F6D40120002800F0B2
:100C2000A08298F8000080076AD5D9F8100010F06B
:100C30003801D9F828001DD0182908BF5FEA807054
:100C400018D0D8F80C00D9F80010002840D021F0B6
:100C500019010843C9F80000FFF7B2FC054600BFC0
:100C6000D9F80000400727D4FFF7AAFC401B022850
:100C7000F6D91EE0D9F80000400704D5D8F80C00DA
:100C8000002800F05E81D9F80000D8F80C1020F0A0
:100C900019000843C9F80000FFF792FC054600BFA1
:100CA000D9F80000400707D4FFF78AFC401B022850
:100CB000F6D90327002420E0D9F80400D8F8101052
:100CC00020F0FE40012440EA0160C9F8040014E06D
:100CD00021F00100C9F80000FFF772FC054601266B
:100CE000D9F8000010F0040086EA900405D0FFF760
:100CF00067FC401B0328F3D30327002C00F031824C
:100D000098F80000C00656D5D9F8100000F0380158
:100D1000D9F82800082905D0182917D100F00300B8
:100D2000012813D1D9F80000C00503D5D8F81C005C
:100D300080283BD1D9F80C00D8F8201020F07C5046
:100D4000012440EA0160C9F80C0031E0D8F81C0029
:100D50000028D9F8000012D040F08000C9F8000047
:100D6000FFF72EFC054600BFD9F80000C005E1D40E
:100D7000FFF726FC401B0228F6D9032717E020F0D6
:100D80008000C9F80000FFF71BFC0546012600BFE4
:100D9000D9F8000010F4807086EA102408D0FFF71C
:100DA0000FFC401B0328F3D3032701E00127002495
:100DB000002C00F0D68198F8000000071CD498F8A9
:100DC0000000800631D498F80000400745D4D8F8D8
:100DD0002440002C00F09180D9F8100000F0380079
:100DE000182840F08C80012CD9F82810D9F8300050
:100DF00040F0A9800127B4E1D8F814000028D9F800
:100E000074003ED040F00100C9F87400FFF7D8FB31
:100E1000054600BFD9F874008007D0D4FFF7D0FB97
:100E2000401B0228F6D903279BE1D8F818000028B8
:100E3000D9F800004DD040F48050C9F80000FFF709
:100E4000BFFB0546D9F800008004BCD4FFF7B8FB0F
:100E5000401B0228F6D9032783E1D9F8000440F4A7
:100E60008070C9F80004FFF7ABFB0546D9F8000411
:100E7000C0051AD4FFF7A4FB401B6428F6D903274A
:100E80006FE120F00100C9F87400FFF799FB0546F7
:100E9000032700BFD9F8740080077FF590AFFFF7F4
:100EA0008FFB401B0228F5D95BE1D8F808502DB123
:100EB000052D00F08280012D00F08580D9F87000AA
:100EC00020F00100C9F87000D9F8700020F004008B
:100ED0007DE020F48050C9F80000FFF771FB054663
:100EE000032700BFD9F8000080047FF56CAFFFF73F
:100EF00067FB401B0228F5D933E1002731E1D9F81F
:100F0000000020F08070C9F80000FFF759FB022CA8
:100F100005464FF0030709D1D9F80000800178D5C4
:100F2000FFF74EFB401B0228F6D91AE1D9F8000062
:100F3000800140F1E780FFF743FB401B0228F5D911
:100F40000FE10127B6E601F00302D8F828309A42F3
:100F500040F0DA80C1F30511D8F82C20914240F01E
:100F6000D7800146D8F830206FF35F21013A9142D3
:100F700040F0D080C0F34622D8F8341001398A42BC
:100F800040F0CA80C0F30642D8F8381001398A42CE
:100F900040F0C480C0F30660D8F83C1001398842A4
:100FA00040F0BE80D9F83400D8F84810C0F3CC0027
:100FB000814240F0B7800027D3E0D9F8700040F0BC
:100FC0000400C9F87000D9F8700040F00100C9F8B9
:100FD0007000FFF7F5FA002D054641F288344FF016
:100FE000030711D0D9F8700080073FF5F0AEFFF786
:100FF000E7FA401BA042F5D9B3E000BFFFF7E0FAE3
:10100000401BA04200F2AD80D9F870008007F5D4F3
:10101000DDE608F12807D9F8280040F2F3318843CB
:101020008ECF0843591E40EA02104FF47E426FF300
:101030005F21C9F8280002EB47204FF4FE0280B27E
:10104000D8F83C300844D8F8381002EB01414FF092
:10105000FE4201F4FE0102EB0362084402F0FE418D
:101060000844C9F83000D9F82C004FF6F87120F088
:101070000100C9F82C00D9F83400D8F8482088437A
:1010800040EAC200C9F83400D9F82C00D8F8401062
:1010900020F00C000843C9F82C00D9F82C00D8F82F
:1010A000441020F002000843C9F82C00D9F82C00A5
:1010B00040F48030C9F82C00D9F82C0040F40030FE
:1010C000C9F82C00D9F82C0040F48020C9F82C0075
:1010D000D9F82C0040F00100C9F82C00D9F8000024
:1010E00040F08070C9F80000FFF76AFA0446032751
:1010F000D9F80000800109D4FFF762FA001B02282A
:10110000F6D92EE000272CE001272AE0002728E06E
:10111000012726E0012724E0012722E0012720E023
:1011200001271EE0D9F82C0020F00100C9F82C009E
:10113000FFF746FA0546FFF743FAA842FBD0D9F875
:1011400034004FF6F871D8F848208843002740EA69
:10115000C200C9F83400D9F82C0040F00100C9F8E9
:101160002C00F8B201B0BDE8F083000000000000E0
:1011700080B500F0A9F880BDFEE700000000000087
:1011800010B584B00024CDE90244CDE90044FFF756
:10119000BFFA0120ADF8000048F21F70029040F243
:1011A0000110039068460194FFF782FA0420FFF7CC
:1011B000BFFA04B010BD000080B541F2C12043F277
:1011C0009032C0F60000C0F60002002100F0DCF909
:1011D00040F27C01C2F20041086080BD00000000C6
:1011E000FEE7000000000000FEE700000000000035
:1011F00000F007004FF0FF3C80F00703042B28BFEE
:101200000423033838BF00200CFA03F399430CFA87
:1012100000F301FA00F022EA0301084370470000DE
:10122000EFF30980BFF36F8F154B1A681EF0100F94
:1012300008BF20ED108A20E9F04F10602DE9090069
:101240004FF0500080F31188BFF34F8FBFF36F8FC3
:1012500001F0F6F94FF0000080F31188BDE80900B5
:1012600019680868B0E8F04F1EF0100F08BFB0EC26
:10127000108A80F30988BFF36F8F704700BF00BFEB
:1012800074010024000000000000000000000000C5
:10129000074B19680868B0E8F04F80F30988BFF37E
:1012A0006F8F4FF0000080F31188704700BF00BFC0
:1012B000740100240000000080B500F0F9F880BD42
:1012C000012000F01DF9FBE7B0B501380024B4EBB4
:1012D000106F01D00120B0BD4EF210050F21CEF2EB
:1012E000000568604FF0FF3000F0CEF8AC600720DA
:1012F00028602046B0BD000080B5FFF769F901F015
:10130000DBFD012808BF80BD01F076FA80BD00003A
:10131000B0B59CB044F6180409A84C21C5F60204E7
:10132000FFF795F802200025CDE90755CDE90555D1
:10133000CDE90355CDE90155FFF736FA00950121B6
:10134000206861F38F302060206800F440400090F6
:10135000009800BF20688004FCD50220099001207D
:101360000C9040200D9009A800241294FFF7F0FB88
:1013700080B93F200121CDE9010401A8CDE9034452
:10138000CDE90544CDE90744FFF732FA002804BF50
:101390001CB0B0BDFFF7FCF84EF6885042F2000CCE
:1013A000CEF20000C5F2002C026842F47002026026
:1013B000DCF8000000F00F00062806D8DCF800007A
:1013C000072262F30300CCF8000044F200404EF61E
:1013D0007F51C5F60200CEF6F621026842F0010206
:1013E000026000220261036819400160DCF800100D
:1013F000090706D5DCF80010072363F30301CCF8D6
:10140000001040F200218261C261C0F2022102623A
:1014100081620021C0F2FF11C16240F28021C0F25E
:101420000111016342638163C26301644264016824
:1014300021F4802101600266D0F8D410C90448BFAD
:101440007047D0F8D41043F2D20241F48051C0F872
:10145000D41044F20001C5F200210A60D0F8D41083
:1014600021F48051C0F8D410704700000000000043
:10147000FEE70000000000004EF60C50CEF2000027
:101480000068C0F3022070474EF6145300F00F02BC
:10149000CEF20003B0F1FF3F1A4400F16043C8BF31
:1014A00003F564420801107070470000000000005E
:1014B0004EF61F500021CEF2000001707047000070
:1014C0004EF60C514FF6FF03CEF200010A681A40A7
:1014D00060F30A2242F0806040F0FD7008607047BF
:1014E000FFF74EFEFFF784F8FFF712FF00F018F841
:1014F000FFF762FE00F02CF8FEE70000000000009D
:10150000EFF3058100291CBF6FF00500704720B183
:1015100080B500F0B9FF002080BD002070470000BA
:10152000EFF3058000281CBF6FF00500704740F204
:101530007800C2F20040016800291CBF4FF0FF3064
:10154000704701210160002070470000000000008A
:1015500010B5EFF3058000281CBF6FF0050010BD2B
:1015600040F27804C2F200442068012807D1FFF756
:10157000A3FE0220206001F007F8002010BD4FF00C
:10158000FF3010BD0000000070B584B08E4600280A
:101590004FF000010391EFF3058146D0002944D1BB
:1015A000FAB19369002B08BF1823382B16D811798C
:1015B000C90713D1556994684FEA950C002D08BFEF
:1015C0004FF0800C1168FCB1D6685C2E1BD3D5B1EE
:1015D0001569C5B10024012555B91BE0002004B0F0
:1015E00070BD0124002118234FF0800C00258DB11F
:1015F000946812690294CDE900326246734601F0A4
:101600001BFC039011E00CB9D4689CB100250024A8
:10161000002DEDD14CB11FFA8CF2009303AB019376
:10162000734601F0D5FB012802D1039804B070BDC8
:101630000020E6E71469B4FA84F46409D6E70000F0
:10164000F0B581B040F6C05240F27416C2F20042CA
:10165000C2F2004604460D4617683268101D00F0BD
:101660007FFD601C0AD14DB13068011D40F69850D5
:10167000C2F2004000F0DCFD01B0F0BD3068E419BA
:1016800044600AD340F28410C2F20040006831681E
:10169000043100F0ADFD01B0F0BD40F27C10C2F2AB
:1016A000004000683168043100F0A2FD40F624508B
:1016B000C2F2004001688C4238BF046001B0F0BD46
:1016C00070B5044600F0D0FD40F2F85040F27415B9
:1016D000C2F20040C2F2004540F68C560168C2F2E8
:1016E000004601310160296841B1306860B928685D
:1016F000E16AC06A884298BF2C6005E02C600068EF
:10170000012801D100F0D4F940F20460C2F2004097
:10171000016801310160616440F20861C2F2004178
:10172000E06A0A68904288BF086000EB800040F2DF
:101730008C11C2F2004101EB8000211D00F078FD08
:1017400000F0BAFD306880B12868E16AC06A88425A
:1017500028BF70BD4EF604504FF08051CEF200000D
:101760000160BFF34F8FBFF36F8F70BD00000000AB
:1017700070B582B000F078FD40F6C456C2F2004663
:10178000306850BB40F6C444C2F20044204600F02A
:101790001FFD40F6D845C2F20045284600F018FD6E
:1017A00040F2781040F28002C2F2004040F2201372
:1017B000C2F20042C2F20043046040F28810C2F25A
:1017C0000040102105600A200025009501F02CF84A
:1017D000306010B103A100F01FFE00F06DFD02B0FB
:1017E00070BD00BF546D7251000000000000000089
:1017F000F0B581B040F2FC55C2F200452868E0B176
:1018000040F6AC5640F2F857C2F20046C2F200472A
:1018100000F02AFDF068C468201D00F0A1FC3868C3
:101820000138386028680138286000F045FD2046FE
:1018300000F05AF828680028EAD101B0F0BD000095
:1018400080B5026C002A08BF80BDD0E902C31344F2
:10185000C360634501D30368C360C3680846194683
:10186000FEF7A8FD80BD000070B5866B0446036CD2
:10187000E3B115461AB3E0681A46FEF79BFDE1682E
:10188000206C2268091A9142E16003D24042A168AB
:101890000844E060A81E3146B0FA80F0002E18BF60
:1018A0000121400900250840361A18E0206800256B
:1018B000A8B9A06801F0C8FBA56005460FE0606804
:1018C0001A46FEF777FD216CD4E9010208446060F6
:1018D000904201D2002502E0206860600025701C63
:1018E000A063284670BD000010B5044690F859006A
:1018F000022808D0012803D030B9206B00F0F4FC96
:10190000204600F0F1FC10BD4FF0500080F311882C
:10191000BFF36F8FBFF34F8FFEE7000000000000A2
:1019200040F27811C2F2004109680A68B2FA82F303
:10193000002A4FEA531202600EBF0020C8680068F8
:10194000704700000000000040F2000040F2801CE0
:10195000C2F20000C2F2004CC11D10F0070221F0DB
:101960000701A0EB010318BF08464FF47051002A8D
:1019700018BF03F5705140F6905200230144C2F2A3
:101980000042083921F00701CCF8001010605360C4
:10199000C1E90033091A4160DCF80020026040F61A
:1019A0002050C2F20040016040F61850C2F20040E0
:1019B000016040F6EC40C2F2004001210170704726
:1019C00040F28C144EF60455C2F20044CEF20005EB
:1019D0004FF08056FFF70CFF20680228FAD32E60E4
:1019E000BFF34F8FBFF36F8FF4E7000000000000DC
:1019F000B0B51C46049D09B12A6000E02D60C5E920
:101A00000F010121284600F05BFF85F84C40B0BD76
:101A10002DE9F0470A9C16460F468246206B91003E
:101A2000A5229846DDE90859FEF709FD206B00EB79
:101A30008600A0F1040020F007067FB104F1340015
:101A4000002100BF7A5C42547A5C1AB10F2901F17F
:101A50000101F7D3002084F8430002E0002084F85D
:101A60003400372D04F1040028BF37250027E56234
:101A7000C4E9135700F0B8FB04F1180000F0B4FB00
:101A8000C5F13800A0613046514642462461646287
:101A9000676584F8587000F04BFBB9F1000F2060C7
:101AA00018BFC9F80040BDE8F08700000000000042
:101AB000B0B540F28C150024C2F20045281900F0A0
:101AC00087FB1434B4F58C6FF8D140F6F044C2F2C1
:101AD0000044204600F07CFB40F60455C2F200456D
:101AE000284600F075FB40F63850C2F2004000F086
:101AF0006FFB40F6AC50C2F2004000F069FB40F6CC
:101B00009850C2F2004000F063FB40F27C10C2F239
:101B10000040046040F28410C2F200400560B0BD95
:101B200040F69052C2F20042114612688242FBD344
:101B3000D1F804C001EB0C03834203D14068604438
:101B400048600846D0F804C000EB0C03934201D073
:101B500013460AE040F28013C2F200431B689A4227
:101B600003D0D2E90032624442608142036018BF70
:101B7000086070470000000080B58C46014694451F
:101B8000006141F804CF08D99A4201D29C4511D294
:101B900040F27810C2F2004007E0D21A8069824217
:101BA00008D240F28810C2F20040006800F020FB2A
:101BB000002080BD012080BD10B5044600F054FB1C
:101BC000A06BB0FA80F0440900F076FB204610BD0F
:101BD00010B5044600F048FBA06BE16B401AB0FA68
:101BE00080F0440900F068FB204610BD00000000B2
:101BF00008480068006880F308884FF0000080F310
:101C0000148862B661B6BFF34F8FBFF36F8F00DFEA
:101C100000BF00BF08ED00E070B582B040F278125E
:101C20000546C2F200420E461268D268D468201DF2
:101C300000F096FA94F82800410704D400F0FE0062
:101C400084F8280010E0A0693246411920462B464E
:101C5000FFF792FF40B100210023002000902046B2
:101C60002A4601F04DFB20B1216A2046884702B088
:101C700070BD4FF0500080F31188BFF36F8FBFF33A
:101C80004F8F00BFFEE700002DE9F04186B040F61F
:101C9000C45702A9C2F2004700224FF0000838687A
:101CA00000F08EFF00286AD001AC02AD0BE000F01E
:101CB000FE0086F8280000BF38680022294600F0A0
:101CC0007FFF00285BD00298B0F1FF3F03DCDDE925
:101CD00003200599904702980028EDD4049E70696E
:101CE00010B1301D00F03CFA204600F0B5F8029922
:101CF0000929E1D80246DFE801F0080808052A3979
:101D00000808052A96F82800D1E796F82800039BD2
:101D1000B16940F0010086F8280019443046FFF709
:101D20002BFF0028C8D0316A3046884796F8280033
:101D30004007C1D50398B1690A1800210023304635
:101D4000CDF8008001F0DCFA0028B5D123E096F848
:101D5000280040F00101039886F82810B06188B18E
:101D6000811830461346FFF707FFA5E796F82800CD
:101D700081073FF59CAF304600F0B6FA9CE706B00D
:101D8000BDE8F0814FF0500080F31188BFF36F8FF2
:101D9000BFF34F8FFEE74FF0500080F31188BFF381
:101DA0006F8FBFF34F8F00BFFEE700000000000001
:101DB00070B582B00E46044600F03AFC01A800F06F
:101DC0004BF8019919B101F0D3F902B070BD054685
:101DD0004EB9A54207D301F0CBF920462946FFF7BB
:101DE0001BFF02B070BD4EB140F28810C2F200403D
:101DF00000680068B0FA80F0420900E0002240F676
:101E0000C450611BC2F20040006800F019FB01F0F1
:101E1000AFF90028D9D14EF604504FF08051CEF2E0
:101E200000000160BFF34F8FBFF36F8F02B070BD32
:101E300040F27C10C2F200400168096821B10068DC
:101E4000C068C068406801E04FF0FF3040F62451A0
:101E5000C2F200410860704770B5044601F040F8D6
:101E600040F270160546C2F200463168884203D23D
:101E700000F00AF8012000E00020206028463560CC
:101E800070BD0000000000002DE9F04182B040F27A
:101E90007817C2F200473868016891B34FF0000824
:101EA00009E000BF606038683146246100F0A0F9A5
:101EB0003868016829B3C068C4680568261D3046C3
:101EC00000F04EF9216A2046884794F82800400720
:101ED000EED5A0692844A842E4D80021002320467A
:101EE0002A46CDF8008001F00BFA0028E0D14FF02F
:101EF000500080F31188BFF36F8FBFF34F8F00BF87
:101F0000FEE740F28811C2F200410A683A600860B8
:101F100002B0BDE8F081000081B00020009040F2E6
:101F20001000C2F2004000684FF0500181F31188A8
:101F3000BFF36F8FBFF34F8F013001D0FEE700BFBB
:101F400000980028FCD001B070470000000000009D
:101F500082B001AC2046FFF7E3FC0199FFF728FFB0
:101F6000FFF792FEF6E70000F0B581B0044600F0FE
:101F70007BF994F94560012E10DB04F1240503E0A0
:101F800070B2013E012809DD286838B1284601F009
:101F9000A7F80028F4D000F0B3FAF1E7FF2684F8A0
:101FA000456000F089F900F05FF994F94470012F61
:101FB00010DB04F1100503E078B2013F012809DDD0
:101FC000286838B1284601F08BF80028F4D000F0DA
:101FD00097FAF1E784F8446000F06EF901B0F0BDC3
:101FE0002DE9F04381B0044600F022FB40F2801658
:101FF000C2F20046306808B9FFF7A6FC40F6EC498B
:10200000C2F2004999F80000002818BF4FF00040C4
:1020100020420ED0002401F0ABF860071FD04FF033
:10202000500080F31188BFF36F8FBFF34F8F00BF55
:10203000FEE7C4B114F0070004F108011EBF081A3E
:1020400000F108015FEA41700ED04FF0500080F3BC
:102050001188BFF36F8FBFF34F8F00BFFEE720469D
:1020600001B0BDE8F083002140F618584A1EC2F2C4
:102070000048D8F800008242CCD240F69050C2F21C
:10208000004005682F4657F8042F8A4211D22B686A
:102090005BB100BF1F4628461D4657F8042F8A42F1
:1020A00007D22B68002BF5D103E040F69050C2F226
:1020B000004033689D42ADD0521A0468112A2B6843
:1020C000036010D36818430709D04FF0500080F325
:1020D0001188BFF36F8FBFF34F8F00BFFEE74260E1
:1020E0003960FFF71DFD40F620503968C2F200400C
:1020F000D8F80020511AC8F800100268083491423C
:1021000038BF016099F80000396800284FF00000DE
:1021100018BF41F000412860396040F62C51C2F2EE
:10212000004108680130086075E700000000000009
:1021300041F6197321F00101C0F6000340F80C3C90
:102140004FF0807340F8202C40E902136FF0020139
:1021500040F8241CA0F1440108467047000000002C
:10216000D0E9013201699A60D0F808C04A68824219
:102170004FF00002CCF8043008BFC1F804C002617F
:102180000868013808600868704700000000000017
:1021900040F60C03C2F20043036040F20C60C2F24E
:1021A00000400860802010607047000000000000C0
:1021B00040F66843C2F20043036040F66800C2F292
:1021C000004008604FF4807010607047000000000D
:1021D00002464FF0FF3142F8081F00214260C0E97B
:1021E0000322016070470000002101617047000078
:1021F00080B5D1F800C01CF1010207D000F108033E
:102200009E465B681A686245FAD901E0D0F810E092
:10221000DEF804204A60CEF804109160C1F808E0AE
:10222000086101680131016080BD0000000000000C
:10223000D0F800C043684B609A688A609A689960D9
:10224000086151600CF1010101607047000000005D
:10225000DFF80C00016841F470010160704700BFB5
:1022600088ED00E0000000004FF0500080F311887E
:10227000BFF36F8FBFF34F8F40F21000C2F20040E8
:102280000168002901F10101016000D070474EF69C
:102290000450CEF200000068000608BF70474FF0FF
:1022A000500080F31188BFF36F8FBFF34F8F00BFD3
:1022B000FEE700000000000040F21000C2F2004003
:1022C000016839B10139016018BF7047002080F3FF
:1022D000118870474FF0500080F31188BFF36F8F63
:1022E000BFF34F8FFEE70000B0B5002808BFB0BDB8
:1022F000044640F6EC40C2F200400078002818BFC7
:102300004FF0004054F8041C08420CD0A4F108051A
:102310002A6892B14FF0500080F31188BFF36F8F9D
:10232000BFF34F8FFEE74FF0500080F31188BFF3EB
:102330006F8FBFF34F8F00BFFEE721EA000044F824
:10234000040C00F075F940F6185054F8041CC2F261
:1023500000400268114401602846FFF7E1FB40F6A7
:102360003050C2F2004001680131016000F000FF0E
:10237000B0BD0000000000004EF210000021CEF2BF
:10238000000044F6D352C1F262020160816040F263
:102390000001C2F200410968A1FB02124FF0FF31B7
:1023A00001EB9211416007210160704700000000BD
:1023B000EFF30580102814D34EF2F03140F2EC52C6
:1023C000CEF20001C2F20042405C1178884208D28D
:1023D0004FF0500080F31188BFF36F8FBFF34F8F22
:1023E000FEE74EF60C5040F2F051CEF20000C2F281
:1023F00000410068096800F4E060884298BF7047B7
:102400004FF0500080F31188BFF36F8FBFF34F8FF1
:10241000FEE700000000000040F64C5C0022C2F223
:10242000004C00BF5CF832301BB10132082AF9D1F0
:1024300070470CEBC2034CF8321058607047000034
:1024400070B515460E460446FFF70EFF94F844009B
:10245000FF2802D1002084F8440094F84500FF28AA
:1024600002D1002084F84500FFF726FFA06B28B9B1
:1024700004F1240031462A4600F066F82046FFF7B2
:1024800073FD70BD0000000010B5D8B1044640F2E5
:102490000060C2F20040006848B14FF0500080F385
:1024A0001188BFF36F8FBFF34F8F00BFFEE700F0BF
:1024B000BFF800212046FFF7C3F800F059FE0028BE
:1024C00018BF10BD4EF604504FF08051CEF2000000
:1024D0000160BFF34F8FBFF36F8F10BD000000008E
:1024E00040F62851C2F200410968016040F6C0512F
:1024F000C2F200410968416070470000000000001E
:1025000040F6CC500121C2F200400160704700004B
:1025100010B568B10C4640F27411C2F2004109686E
:102520001831FFF765FE01212046FFF789F810BD3D
:102530004FF0500080F31188BFF36F8FBFF34F8FC0
:10254000FEE7000000000000B0B590B10D4640F27B
:102550007411C2F20041144609681831FFF768FE91
:10256000002C214618BF4FF0FF352846FFF768F8CA
:10257000B0BD4FF0500080F31188BFF36F8FBFF3F1
:102580004F8F00BFFEE7000010B586B005A804A974
:1025900003AA0024CDE90444FFF7FAFDDDE9032096
:1025A00005990023CDE9010141F6C1101DA1C0F636
:1025B0000000009400F040FC40F61C51C2F20041C3
:1025C000086010B100F060FE0446601C20D0012CB1
:1025D0001CD14FF0500080F31188BFF36F8FBFF311
:1025E0004F8F40F62450C2F200404FF0FF3101609F
:1025F00040F68C50C2F200400121016040F6C0500C
:10260000C2F200400021016000F06AF806B010BD7F
:102610004FF0500080F31188BFF36F8FBFF34F8FDF
:10262000FEE700BF49444C450000000000000000E8
:1026300040F20060C2F20040016801310160704761
:1026400040F20060C2F20040006830B140F6CC5069
:102650000121C2F200400160704740F6CC5040F2C8
:10266000086CC2F20040C2F2004C002140F28C1211
:102670000160C2F20042DCF8001001EB810352F865
:10268000230048B902EB8300A0F11403D9B153F839
:10269000140901390028F9D001EB810002EB800216
:1026A00052F8040F4368101D8342136001D158682B
:1026B0001060106840F27412C2F20042C0681060EC
:1026C000CCF8001070474FF0500080F31188BFF332
:1026D0006F8FBFF34F8F00BFFEE7000000000000C8
:1026E00080B582B04EF200404CF27021CEF2000074
:1026F000C4F20F114B1CD0F800299A4209D14FF0B7
:10270000500080F31188BFF36F8FBFF34F8F00BF6E
:10271000FEE7D0F800298A4209D14FF0500080F33B
:102720001188BFF36F8FBFF34F8F00BFFEE70178B3
:1027300040F2EC520191FF210170C2F20042017897
:102740008DF803109DF8031001F05001117040F254
:10275000F0510722C2F200410A609DF90320B2F154
:10276000FF3F0CDC0A6800BF9DF80330013A5B00B4
:102770008DF803309DF90330002BF5D40A600A6808
:10278000032A2DD14FF4E06303EA02220A60019983
:102790000170D0F8201941F47001C0F82019D0F868
:1027A000201941F07041C0F82019FFF7E5FD40F213
:1027B00010000021C2F200400160FFF749FD4EF613
:1027C0003470CEF20000016841F040410160FFF733
:1027D0000FFAFFF735FFFFF79FFB002002B080BD27
:1027E0004FF0500080F31188BFF36F8FBFF34F8F0E
:1027F000FEE700000000000080B54FF0500080F3BD
:102800001188BFF36F8FBFF34F8F00F071FB30B1B2
:102810004EF604504FF08051CEF2000001600020CF
:1028200080F3118880BD0000B0B582B068B11D464C
:10283000ABB1F1B9EAB14FF0500080F31188BFF3AA
:102840006F8FBFF34F8F00BFFEE74FF0500080F354
:102850001188BFF36F8FBFF34F8F00BFFEE74FF0BC
:10286000500080F31188BFF36F8FBFF34F8F00BF0D
:10287000FEE751B14AB94FF0500080F31188BFF321
:102880006F8FBFF34F8F00BFFEE750230193019B73
:10289000502B0AD1069B019C012485F846400095E7
:1028A000FFF7A6F8284602B0B0BD4FF0500080F305
:1028B0001188BFF36F8FBFF34F8F00BFFEE700009B
:1028C00070B500B304460E46FFF7CEFCD4E90F0105
:1028D0002268002501FB0023013800FB0120A563CD
:1028E0006260C4E902304FF0FF0084F8440084F8CD
:1028F000450004F1100086B1FFF76AFC04F12400E2
:10290000FFF766FC19E04FF0500080F31188BFF329
:102910006F8FBFF34F8F00BFFEE7016869B100F012
:10292000DFFB50B14EF604504FF08051CEF2000064
:102930000160BFF34F8FBFF36F8FFFF7BDFC012026
:1029400070BD0000000000002DE9F04F83B002923E
:10295000B8B104461D460E46E9B1022D03D1E06B25
:10296000012840F09A8000F0A7FA00BB0298F0B16D
:102970004FF0500080F31188BFF36F8FBFF34F8F7C
:10298000FEE74FF0500080F31188BFF36F8FBFF365
:102990004F8F00BFFEE7206C0028DED04FF05000C4
:1029A00080F31188BFF36F8FBFF34F8FFEE7FFF700
:1029B0005BFC022DA06B58D0E16B884255D304F12B
:1029C000100801206F464FF0000B0DF108094FF081
:1029D000805A00BF0299002900F07B80C00702D016
:1029E0003846FFF77DFDFFF767FCFFF721FEFFF795
:1029F0003BFC94F84400FF2808BF84F844B094F8E6
:102A00004500FF2808BF84F845B0FFF755FC38465D
:102A1000494600F099F900285ED12046FFF7D8F822
:102A2000A0B102994046FFF773FD2046FFF79CFADC
:102A300000F09EFB78B94EF60450CEF20000C0F8CC
:102A400000A0BFF34F8FBFF36F8F04E02046FFF766
:102A50008BFA00F08DFBFFF707FC022DA06B04D072
:102A6000E16B88424FF00000B4D2204631462A463E
:102A7000FEF7FAFE54F8241FC9B1204600F030FBDF
:102A800008B34EF604504FF08051CEF200000160C2
:102A9000BFF34F8FBFF36F8F15E04FF0500080F3FF
:102AA0001188BFF36F8FBFF34F8F00BFFEE750B1A8
:102AB0004EF604504FF08051CEF200000160BFF39B
:102AC0004F8FBFF36F8FFFF7F7FB012003B0BDE817
:102AD000F08FFFF7F1FB04E02046FFF745FA00F026
:102AE00047FB002003B0BDE8F08F000000000000AD
:102AF0002DE9F04381B0E8B105461E4691460F46E8
:102B000009B3022E02D1E86B012837D1FFF750FC40
:102B1000EFF311884FF0500080F31188BFF36F8FEF
:102B2000BFF34F8F022EA86B19D0E96B884216D3E2
:102B300000203EE04FF0500080F31188BFF36F8F0C
:102B4000BFF34F8FFEE7286C0028DAD04FF050001B
:102B500080F31188BFF36F8FBFF34F8FFEE795F8B7
:102B60004540A86B284639463246FEF77DFEFF2CCD
:102B70000DD0601C85F8450001201AE04FF0500090
:102B800080F31188BFF36F8FBFF34F8FFEE755F8C7
:102B9000240F68B1284600F0A3FA01460120B9F1DC
:102BA000000F18BF002904D00120C9F8000000E080
:102BB000012088F3118801B0BDE8F0830000000017
:102BC0002DE9F04F85B0049298B104460D460029D6
:102BD00000F0A58000F070F9A8B9049898B14FF002
:102BE000500080F31188BFF36F8FBFF34F8F00BF8A
:102BF000FEE74FF0500080F31188BFF36F8FBFF3F3
:102C00004F8F00BFFEE704F1100904F1240001908A
:102C100002AF0DF1100A4FF000080AE02046FFF75E
:102C2000A3F900F0A5FA2046FEF7C6FF002840F001
:102C30008480FFF719FBD4F838B0BBF1000F1DD02A
:102C400020462946FEF7FCFDABF10100A063206998
:102C500070B1484600F044FA50B14EF604504FF0BF
:102C60008051CEF200000160BFF34F8FBFF36F8F32
:102C7000FFF722FB00200126A0B95FE0049850B1C5
:102C8000B8F1000F02D13846FFF72AFC4FF00108D7
:102C9000012038B952E0FFF70FFB00260020002882
:102CA0004CD000BFFFF708FBFFF7C2FCFFF7DCFAD0
:102CB00094F84400FF2802D1002084F8440094F8DE
:102CC0004500FF2802D1002084F84500FFF7F4FA00
:102CD0003846514600F038F800289FD12046FEF7CC
:102CE0006BFFB0B104990198FFF712FC2046FFF783
:102CF0003BF900F03DFA00289BD14EF604504FF00E
:102D00008051CEF200000160BFF34F8FBFF36F8F91
:102D10008FE72046FFF728F900F02AFA89E7206CB0
:102D200000283FF457AF4FF0500080F31188BFF3F5
:102D30006F8FBFF34F8F00BFFEE70026304605B010
:102D4000BDE8F08F00000000B0B5D0B10D4611B362
:102D50000446FFF789FA40F6C050C2F2004001680D
:102D60002868421C21D040F628536268C2F2004312
:102D70009142D3F800C01AD323689C4517D0012490
:102D800022E04FF0500080F31188BFF36F8FBFF344
:102D90004F8F00BFFEE74FF0500080F31188BFF364
:102DA0006F8FBFF34F8F00BFFEE700240CE0891A3E
:102DB000884206D9401A28602046FFF791FB00247C
:102DC00002E0012400202860FFF776FA2046B0BD1B
:102DD0002DE9F04383B00746900098461546894692
:102DE000FFF7FEF878B106465C20FFF7F9F838B136
:102DF0000446066354B94FF0FF3003B0BDE8F083DA
:102E00003046FFF771FA0024002CF4D0DDE90A10F7
:102E1000002284F85920CDE90010384649462A4658
:102E200043460294FEF7F4FD2046FEF749FC0120DC
:102E300003B0BDE8F083000070B586B00B9CD4B140
:102E40000C9E16B35C250495049D5C2D27D1DDF8FE
:102E500028C0049D3463022586F85950CDF800C07F
:102E600005ADCDE90156FEF7D3FD3046FEF728FC4F
:102E7000059806B070BD4FF0500080F31188BFF385
:102E80006F8FBFF34F8F00BFFEE74FF0500080F30E
:102E90001188BFF36F8FBFF34F8F00BFFEE74FF076
:102EA000500080F31188BFF36F8FBFF34F8F00BFC7
:102EB000FEE700000000000040F68C50C2F2004027
:102EC000006848B140F20060C2F200400068B0FA09
:102ED00080F040094000704701207047000000006A
:102EE00040F6C050C2F20040006870470000000089
:102EF0002DE9F04F81B040F20060C2F2004000685E
:102F000040B140F634500024C2F200400168013163
:102F1000016092E040F6C050C2F2004001684E1CD1
:102F2000066021D340F27C10C2F2004001680968BB
:102F300049B14FF0500080F31188BFF36F8FBFF39A
:102F40004F8F00BFFEE740F284120168C2F20042D8
:102F50001368036040F628501160C2F20040016817
:102F600001310160FEF764FF40F6245140F2741A0B
:102F7000C2F2004140F28C18C2F2004AC2F200488C
:102F80000868864201D2002445E040F27C17002404
:102F9000C2F200473868006898B340F2086BC2F28A
:102FA000004B19E0D9F82C00DBF8001088422946C4
:102FB00088BFCBF8000000EB800008EB8000FFF733
:102FC00037F9D9F82C00DAF80010C96A3A68884253
:102FD00028BF01241068B8B13868C068D0F80C90D8
:102FE0004D4655F8040F864210D32846FFF7B8F82F
:102FF000D9F828000028D5D009F11800FFF7B0F85B
:10300000D0E74FF0FF3005E04FF0FF3040F624519D
:10301000C2F200410860DAF80000C06A00EB8000EC
:1030200058F82000012840F6CC50C2F2004088BF7A
:1030300001240068002818BF0124204601B0BDE823
:10304000F08F000000000000B0B580B1044640F2EF
:103050007410C2F200400068A0420AD04FF0500045
:1030600080F31188BFF36F8FBFF34F8FFEE700200F
:10307000B0BD206D38B3013820654FF0000021D17C
:10308000E16AE26C914208BFB0BD251D2846FFF7FA
:1030900067F8E06CE062C0F13801A16140F20861BC
:1030A000C2F200410A68904288BF086000EB8000CD
:1030B00040F28C11C2F2004101EB80002946FFF77B
:1030C000B7F80120B0BD4FF0500080F31188BFF376
:1030D0006F8FBFF34F8F00BFFEE7000000000000BE
:1030E000B0B5C068C5687DB105F118042046FFF78A
:1030F00037F840F20060C2F20040006868B140F664
:103100003850C2F200401DE04FF0500080F31188AB
:10311000BFF36F8FBFF34F8FFEE72C1D2046FFF7E5
:103120001FF840F20861E86AC2F200410A68904262
:1031300088BF086000EB800040F28C11C2F20041B1
:1031400001EB80002146FFF773F840F27410E96A42
:10315000C2F200400068C06A814206D940F6CC51F4
:103160000120C2F200410860B0BD0020B0BD0000E7
:103170002DE9F04F81B040F20064C2F200442068B3
:1031800068B1FFF771F8206801382060206880B1CD
:103190000024FFF791F8204601B0BDE8F08F4FF012
:1031A000500080F31188BFF36F8FBFF34F8F00BFC4
:1031B000FEE740F2F850C2F20040006800285DD0FF
:1031C00040F6385640F6CC58C2F20046C2F20048EB
:1031D000306888B340F2086740F28C1940F2741BE3
:1031E000C2F20047C2F20049C2F2004B4FF0010A9E
:1031F000F068C56805F11800FEF7B2FF2C1D2046E7
:10320000FEF7AEFFE86A39688842214688BF386019
:1032100000EB800009EB8000FFF70AF8E86ADBF8B2
:103220000010C96A884228BFC8F800A0306800288A
:10323000DED10DB1FEF7FCFD40F63454C2F200447D
:1032400025685DB1012600BFFFF752FE002818BFB8
:10325000C8F80060013DF7D100202060D8F80000D8
:1032600070B14EF604504FF08051CEF200000124B0
:103270000160BFF34F8FBFF36F8F8AE7002488E7A9
:10328000002486E70000000080B586B0FEF770FAE3
:1032900040F6C450C2F20040006808B3002004A900
:1032A000CDE9040005A803AAFEF782FFDDE90320AB
:1032B00002210023CDE9001041F651700DA1C0F6A6
:1032C0000000DDF814C0CDF808C0FFF7B5FD40F6EA
:1032D000C851C2F20041086010B1012006B080BDA3
:1032E0004FF0500080F31188BFF36F8FBFF34F8F03
:1032F000FEE700BF546D72205376630000000000AB
:1033000010B584B0A0B140F6C4548646C2F2004461
:103310002068B0B10529CDF808E0CDE9001213DC32
:10332000FFF7CAFD0228206816D1069A694615E003
:103330004FF0500080F31188BFF36F8FBFF34F8FB2
:10334000FEE7002004B010BD9C466946002362469B
:10335000FFF7CEFB04B010BD694600220023FFF743
:10336000F3FA04B010BDF1EE100A4FF6FF71C0F28F
:10337000C03120EA010040F04070E1EE100A7047D1
:10338000000000000102030401020304060708090B
:10339000B43300080000000000000000000000003E
:1033A0000000000000020000180000000000000003
:1033B0000000000064656661756C745461736B0095
:1033C000F033000800000024180000000803000883
:1033D000F033000800000020003C00002403000837
:1033E0000834000818000024B81300002403000863
:1033F0000090D0030090D0030100000010000000F6
:08340000AAAAAAAA000000001C
:04000005080002CD20
:00000001FF
